:020000040000FA
:0400000080313428EF
:080008008031332882073F34E8
:1000100006345B344F3466346D347D3407347F34BA
:100020006F34403476341030AA00A201A3010310CB
:10003000A60DA70D0310A00DA10DA20DA30D230861
:100040002502031D25282208240203192928031844
:1000500030282508A3022408A202031CA3032614A7
:10006000AA0B172808009128210099178730190535
:1000700050389900FC3099053F3024008C003F3007
:100080008E002100951323008C018E0121009D011B
:100090009E012200910192019301940121008C158F
:1000A0000E108E100E118E110C110C128C128E125D
:1000B0000E12E1302000AC00AC30AD00813142299D
:1000C00022008E118E1040302000AF004030B00072
:1000D0004030B1004030B2004030B3001C118730D6
:1000E0009C05FC309C050E309B009A01210091106C
:1000F0000B1720001C1524009512F030150503384D
:100100009500151214172000AE01911122008E15D2
:1001100024009516210091150B178B1724009101CF
:1001200008002000911DEC282E08031DA5282200A0
:100130000E128E140C15200030082400910001309E
:100140002000AE0022008E10EA282E03031DB628E0
:1001500022000C118E140C1620003108240091008E
:1001600002302000AE0022008E10EA2802302E025B
:10017000031DC82822000C128E148C162000320891
:100180002400910003302000AE0022008E10EA28E7
:1001900003302E02031DDA2822008C128E148E16D4
:1001A000200033082400910004302000AE0022001B
:1001B0008E10EA2804302E02031DEA2822008E1237
:1001C0008E140E1620002F08240091002000AE018E
:1001D00022008E102000911109007630AF00763099
:1001E000B0007630B1007630B2007630B30008004F
:1001F00003102D0CBE002C0CBD000310BE0CBD0C5A
:100200003D082C06BF003E082D06C00003102D0C33
:10021000C2002C0CC1000310C20CC10C0310C20C94
:10022000C10C41083F06C30042084006C400031049
:100230002D0CC6002C0CC5000430A0000310C60C09
:10024000C50C8131A00B1E2945084306C70046088E
:100250004406C80001304705BB00BC0103102D0C4B
:10026000BE002C0CBD00BF01C0013B18C0173F08E9
:100270003D04AC0040083E04AD002C08A0002D0851
:10028000A1000800803160203430200098009901DE
:10029000391420006830A0000230A1008131A10B88
:1002A0004F298131A00B4C298031F82020002008F3
:1002B000B6002108B70082318C19452A2000D030C1
:1002C000A0000830A1008131A10B64298131A00B6D
:1002D000612920000130A0008131A00B6D290000B0
:1002E00000008231391C452A39104030AF004030BF
:1002F000B0004030B1004030B2004030B300D030E8
:10030000B6000730B700360837043915031939111C
:1003100081318C1D8D29B9118E29B91539163919DC
:10032000B91D3912391EA12920002830A0008131C1
:10033000A00B982900000000B603360A0319B70382
:100340008329360837048231031D432A8031F8207F
:1003500020002008B6002108B700360837043917F6
:100360000319391381318C1DB729B913B829B9176D
:100370003A14391BB91F3A103A1CCA29200003301D
:10038000A0008131A00BC2290000B603360A031970
:10039000B703AD29360837048231031D3F2A1810F0
:1003A0009601970111107630B100181481318C1923
:1003B000DA29D6291810823111183B2A1608B40000
:1003C0001708B5001030A4002730A5003408A0009D
:1003D0003508A1008031132020002608B8008031A4
:1003E00006202000AF002208B4002308B500E83042
:1003F000A4000330A5003408A0003508A100803116
:10040000132020002608B800803106202000B0000C
:100410002208B4002308B5006430A400A501340804
:10042000A0003508A1008031132020002608B80064
:10043000803106202000B1002208B4002308B50056
:100440000A30A400A5013408A0003508A1008031BD
:10045000132020002608B800803106202000B200BA
:100460002208B4002308B50034088031062020009B
:10047000B3008231452A8031ED208231452A803116
:10048000ED208231452A8031ED20813120008C1D04
:0604900049293914492935
:020000040001F9
:02000E00840963
:02001000FF1ED1
:00000001FF
